:020000020000FC
:0200000069C0D5
:02000C0005C02D
:100016003EC00FB70F93012F0A3018F10F3790F03B
:100026000B38E0F0012F0158000F00950BBD0FEFC4
:100036000ABDAA95A83008F0A7E00C9105BB0F9160
:100046000FBF1895012F0050000F00950BBD0FEF45
:100056000ABDA395A83088F3A0E0EFCF00E005BB6A
:10006600EECF05E00BBD0FEF0ABD761718F0671748
:1000760038F0E5CF7395A395A830F8F2A0E0DDCF70
:10008600AD9A7A95AA95A830C0F2A7E0D6CF4CB122
:100096008BB184FD16C0B89423950BF431E080E053
:1000A60038130EC082E0281307C0142F81E04817CA
:1000B60038F0AD9A000004C083E0281301C0642F15
:1000C60018955498579833272227AC98F9CF04E00F
:1000D6000EBF0FE50DBF9FE794BB90E095BB549A0A
:1000E60090E090BD91E099B993E69BBD9FEB9ABDD8
:1000F60090E09DBD9CBD9FBD90E498BF90E199BFE7
:10010600F1E0E6E5B1E0A0E090E1C8950D92319608
:100116009A95D9F7B1E0A0E09BE09EBD789466275A
:1001260077278099FECF90E18099FBCF9395E3F7EF
:100136005498579833272227AC98AD98809BFECFCA
:100146005F980000AC9A549A579A00000000E9CFD5
:0801560009080C040602030174
:00000001FF
